:020000040000FA
:1000000017EF17F01200FFFFFFFFFFFFFFFFFFFFDB
:10001000FFFFFFFFFFFFFFFFFFFFFFFFFFFFFFFFF0
:10002000FFFFFFFFFFFFFFFFFFFFFFFFFFFFFFFFE0
:10003000FFFFFFFFFFFFFFFFFFFFFFFFFFFFFFFFD0
:10004000FFFFFFFFFFFFFFFFFFFFFFFFFFFFFFFFC0
:1008000017EF17F01200FFFFFFFFFFFFFFFFFFFFD3
:10081000FFFFFFFFFFFFFFFFFFFFFFFFFFFFFFFFE8
:10082000FFFFFFFFFFFFFFFFFFFF01002D2E000076
:10083000F4010000010000000101A66B1200060E89
:100840000101EE5D03E36D50020B02E05EEF0EF07E
:10085000400EE66E000EE66E010EE66E57EC0FF0EF
:10086000E552E552E5520101A36FA35104E15EEFA9
:100870000EF05EEF0EF0A56BA351A55D02E35EEFF7
:100880000EF0A551EA6A000FE96E010EEA22EFCFE1
:10089000A4F1A6510E0A02E1D3EF09F0030A01E127
:1008A000E9D2010A01E1D8D2070A01E1BBD2010A6B
:1008B00001E19ED2030A01E18CD2010A01E17AD260
:1008C0000F0A01E100D2010A01E11ED1030A01E190
:1008D0000CD1010A01E1FAD0070A01E19BD0010A1B
:1008E0003AE0030A1EE0010A02E05BEF0EF0B06B93
:1008F000B16BB26BB36B4D0EA45D06E0450EA45D0B
:1009000003E0440EA45D05E1A4C1A7F1010EA66FAA
:1009100006D00A0EA45D03E00D0EA45D00E05BEFBF
:100920000EF0300EA45D09E3A451390806E3300E41
:10093000A45DA86F020EA66F0CD02A0EA45D08E17C
:10094000B069B169B2693F0EB36F080EA66F01D0EE
:10095000A66B5BEF0EF0300EA45D09E3A4513908DD
:1009600006E3300EA45DA96F030EA66F51D02C0EC6
:10097000A45D1EE1010EA8C1E7FFE75204E0E846CE
:10098000FE0BE706FCE10101B46FB56BB66BB76B0C
:10099000800B03E0B569B669B769B451B013B551BE
:1009A000B113B651B213B751B313040EA66F30D0C2
:1009B0002D0EA45D05E1A8C1AAF1050EA66F28D0F1
:1009C000230EA45D24E1010EA8C1E7FFE75204E075
:1009D000E846FE0BE706FCE10101B46FB56BB66BB0
:1009E000B76B800B03E0B569B669B769B451B01352
:1009F000B551B113B651B213B751B3134D0EA75D34
:100A000003E1090EA66F02D00E0EA66F01D0A66BF1
:100A10005BEF0EF0230EA45D27E10A0EA803F3504E
:100A2000A925146E010E145204E0E846FE0B1406CC
:100A3000FCE10101B46FB56BB66BB76B800B03E0E3
:100A4000B569B669B769B451B013B551B113B651B0
:100A5000B213B751B3134D0EA75D03E1090EA66F94
:100A600002D00E0EA66F30D02C0EA45D21E10A0E2E
:100A7000A803F350A925146E010E145204E0E846B1
:100A8000FE0B1406FCE10101B46FB56BB66BB76BDE
:100A9000800B03E0B569B669B769B451B013B551BD
:100AA000B113B651B213B751B313040EA66F0CD0E5
:100AB0002D0EA45D08E10A0EA803F350A925AA6F24
:100AC000050EA66F01D0A66B5BEF0EF0300EA45D95
:100AD00009E3A451390806E3300EA45DA86F020EA5
:100AE000A66F01D0A66B5BEF0EF0300EA45D09E39C
:100AF000A451390806E3300EA45DA86F060EA66F58
:100B000001D0A66B5BEF0EF0300EA45D09E3A4519B
:100B1000390806E3300EA45DA96F070EA66FD1D089
:100B20002C0EA45D62E1A8C1ABF1AB51D880AA55EF
:100B300005E2AAC1ADF1ABC1ACF104D0ABC1ADF1DE
:100B4000AAC1ACF11468156816681768020EAAC12C
:100B5000E7FFE75204E0E846FE0BE706FCE1FF0F83
:100B6000186E196A1A6A1B6A18AE03D019681A68D7
:100B70001B681850145C0101B86F19501558B96FF3
:100B80001A501658BA6F1B501758BB6F020EABC1E4
:100B9000E7FFE75204E0E846FE0BE706FCE1FF0F43
:100BA0000101BC6FBD6BBE6BBF6B800B03E0BD6909
:100BB000BE69BF69BC0EE96E010EEA6EB851EE1453
:100BC000B46FB951EE14B56FBA51EE14B66FBB5194
:100BD000EE14B76FB451B013B551B113B651B2138F
:100BE000B751B313040EA66F6CD0230EA45D68E159
:100BF000A8C1ABF1AB51D880AA5505E2AAC1ADF1AD
:100C0000ABC1ACF104D0ABC1ADF1AAC1ACF1146879
:100C1000156816681768020EAAC1E7FFE75204E0DC
:100C2000E846FE0BE706FCE1FF0F186E196A1A6A28
:100C30001B6A18AE03D019681A681B681850145C38
:100C40000101B86F19501558B96F1A501658BA6F7C
:100C50001B501758BB6F020EABC1E7FFE75204E011
:100C6000E846FE0BE706FCE1FF0F0101BC6FBD6B20
:100C7000BE6BBF6B800B03E0BD69BE69BF69BC0E74
:100C8000E96E010EEA6EB851EE14B46FB951EE146C
:100C9000B56FBA51EE14B66FBB51EE14B76FB451C5
:100CA000B013B551B113B651B213B751B3134D0EC2
:100CB000A75D03E1090EA66F02D00E0EA66F01D04C
:100CC000A66B5BEF0EF00A0EA803F350A925AB6FDD
:100CD000AB51D880AA5505E2AAC1ADF1ABC1ACF1C8
:100CE00004D0ABC1ADF1AAC1ACF1146815681668A7
:100CF0001768020EAAC1E7FFE75204E0E846FE0BC0
:100D0000E706FCE1FF0F186E196A1A6A1B6A18AE33
:100D100003D019681A681B681850145C0101B86F79
:100D200019501558B96F1A501658BA6F1B501758EA
:100D3000BB6F020EABC1E7FFE75204E0E846FE0BD3
:100D4000E706FCE1FF0F0101BC6FBD6BBE6BBF6B23
:100D5000800B03E0BD69BE69BF69BC0EE96E010E80
:100D6000EA6EB851EE14B46FB951EE14B56FBA51C2
:100D7000EE14B66FBB51EE14B76FB451B013B5514A
:100D8000B113B651B213B751B3132C0EA45D03E1E6
:100D9000040EA66F0DD0230EA45D09E14D0EA75DD4
:100DA00003E1090EA66F02D00E0EA66F01D0A66B4E
:100DB0005BEF0EF0230EA45D09E14D0EA75D03E18C
:100DC000090EA66F02D00E0EA66F01D0A66B5BEFC8
:100DD0000EF0300EA45D09E3A451390806E3A4C166
:100DE0009EF19F6B0A0EA66F01D0A66B5BEF0EF013
:100DF000300EA45D09E3A451390806E3A4C19FF1B4
:100E0000A06B0B0EA66F0CD0250EA45D03E0230E85
:100E1000A45D05E1A4C1AFF10D0EA66F01D0A66BD4
:100E20005BEF0EF0300EA45D09E3A451390806E330
:100E3000A4C1A0F1A16B0C0EA66F0CD0250EA45D71
:100E400003E0230EA45D05E1A4C1AFF10D0EA66F72
:100E500001D0A66B5BEF0EF0250EA45D03E0230E20
:100E6000A45D05E1A4C1AFF10D0EA66F01D0A66B84
:100E70005BEF0EF00A0EA45D04E00D0EA45D01E030
:100E80008ED29E0EE66E010EE66E74EC15F0E55203
:100E9000E552F3CFAEF1250E0101AF5D27E1AE5172
:100EA000640804E2A66B5BEF0EF020D0AEC107F041
:100EB0008BEC13F005C014F006C015F007C016F057
:100EC00008C017F00A6A0B6A200E0C6E400E0D6EF9
:100ED00014C005F015C006F016C007F017C008F0E2
:100EE0009CEC13F009EC14F007C0AEF1B0C114F0A3
:100EF000B1C115F0B2C116F0B3C117F0010E14164E
:100F0000156A166A176A145015101610171002E0A9
:100F1000AEC180F1B0C114F0B1C115F0B2C116F08C
:100F2000B3C117F0020E1416156A166A176A145028
:100F300015101610171002E0AEC181F1B0C114F007
:100F4000B1C115F0B2C116F0B3C117F0040E1416FA
:100F5000156A166A176A145015101610171002E059
:100F6000AEC182F1B0C114F0B1C115F0B2C116F03A
:100F7000B3C117F0080E1416156A166A176A1450D2
:100F800015101610171002E0AEC183F1B0C114F0B5
:100F9000B1C115F0B2C116F0B3C117F0100E14169E
:100FA000156A166A176A145015101610171002E009
:100FB000AEC184F1B0C114F0B1C115F0B2C116F0E8
:100FC000B3C117F0200E1416156A166A176A14506A
:100FD00015101610171002E0AEC185F1B0C114F063
:100FE000B1C115F0B2C116F0B3C117F0400E14161E
:100FF000156A166A176A145015101610171002E0B9
:10100000AEC186F1B0C114F0B1C115F0B2C116F095
:10101000B3C117F0800E1416156A166A176A1450B9
:1010200015101610171002E0AEC187F1B0C114F010
:10103000B1C115F0B2C116F0B3C117F0146A010EB8
:101040001516166A176A145015101610171002E0BC
:10105000AEC188F1B0C114F0B1C115F0B2C116F043
:10106000B3C117F0146A020E1516166A176A1450E7
:1010700015101610171002E0AEC189F1B0C114F0BE
:10108000B1C115F0B2C116F0B3C117F0146A040E65
:101090001516166A176A145015101610171002E06C
:1010A000AEC18AF1B0C114F0B1C115F0B2C116F0F1
:1010B000B3C117F0146A080E1516166A176A145091
:1010C00015101610171002E0AEC18BF1B0C114F06C
:1010D000B1C115F0B2C116F0B3C117F0146A100E09
:1010E0001516166A176A145015101610171002E01C
:1010F000AEC18CF1B0C114F0B1C115F0B2C116F09F
:10110000B3C117F0146A200E1516166A176A145028
:1011100015101610171002E0AEC18DF1B0C114F019
:10112000B1C115F0B2C116F0B3C117F0146A400E88
:101130001516166A176A145015101610171002E0CB
:10114000AEC18EF1B0C114F0B1C115F0B2C116F04C
:10115000B3C117F0146A800E1516166A176A145078
:1011600015101610171002E0AEC18FF1B0C114F0C7
:10117000B1C115F0B2C116F0B3C117F0146A156A07
:10118000010E1616176A145015101610171002E0EB
:10119000AEC190F1B0C114F0B1C115F0B2C116F0FA
:1011A000B3C117F0146A156A020E1616176A1450A6
:1011B00015101610171002E0AEC191F1B0C114F075
:1011C000B1C115F0B2C116F0B3C117F0146A156AB7
:1011D000040E1616176A145015101610171002E098
:1011E000AEC192F1B0C114F0B1C115F0B2C116F0A8
:1011F000B3C117F0146A156A080E1616176A145050
:1012000015101610171002E0AEC193F1B0C114F022
:10121000B1C115F0B2C116F0B3C117F0146A156A66
:10122000100E1616176A145015101610171002E03B
:10123000AEC194F1B0C114F0B1C115F0B2C116F055
:10124000B3C117F0146A156A200E1616176A1450E7
:1012500015101610171002E0AEC195F1B0C114F0D0
:10126000B1C115F0B2C116F0B3C117F0146A156A16
:10127000400E1616176A145015101610171002E0BB
:10128000AEC196F1B0C114F0B1C115F0B2C116F003
:10129000B3C117F0146A156A800E1616176A145037
:1012A00015101610171002E0AEC197F1B0C114F07E
:1012B000B1C115F0B2C116F0B3C117F0146A156AC6
:1012C000166A010E1716145015101610171002E0AA
:1012D000AEC198F1B0C114F0B1C115F0B2C116F0B1
:1012E000B3C117F0146A156A166A020E1716145065
:1012F00015101610171002E0AEC199F1B0C114F02C
:10130000B1C115F0B2C116F0B3C117F0146A156A75
:10131000166A040E1716145015101610171002E056
:10132000AEC19AF1B0C114F0B1C115F0B2C116F05E
:10133000B3C117F0146A156A166A080E171614500E
:1013400015101610171002E0AEC19BF1B0C114F0D9
:10135000B1C115F0B2C116F0B3C117F0146A156A25
:10136000166A100E1716145015101610171002E0FA
:10137000AEC19CF1B0C114F0B1C115F0B2C116F00C
:10138000B3C117F0146A156A166A200E17161450A6
:1013900015101610171002E0AEC19DF100D001012A
:1013A000A66B5BEF0EF00A0EA45D05E00D0EA45DCA
:1013B00002E05AEF0EF0A751440A01E13FD2010AC0
:1013C00002E059EF0EF0B0C114F0B1C115F0B2C196
:1013D00016F0B3C117F0010E1416156A166A176AD3
:1013E000145015101610171001E09290B0C114F0AF
:1013F000B1C115F0B2C116F0B3C117F0010E141649
:10140000156A166A176A145015101610171001E0A5
:101410009292B0C114F0B1C115F0B2C116F0B3C1CF
:1014200017F0010E1416156A166A176A1450151073
:101430001610171001E09294B0C114F0B1C115F06C
:10144000B2C116F0B3C117F0010E1416156A166A70
:10145000176A145015101610171001E09296B0C1BB
:1014600014F0B1C115F0B2C116F0B3C117F0010EFE
:101470001416156A166A176A1450151016101710EC
:1014800001E09298B0C114F0B1C115F0B2C116F0EC
:10149000B3C117F0010E1416156A166A176A1450B4
:1014A00015101610171001E0929AB0C114F0B1C1D6
:1014B00015F0B2C116F0B3C117F0010E1416156A7B
:1014C000166A176A145015101610171001E0939041
:1014D000B0C114F0B1C115F0B2C116F0B3C117F02C
:1014E000010E1416156A166A176A14501510161094
:1014F000171001E09392B0C114F0B1C115F0B2C160
:1015000016F0B3C117F0010E1416156A166A176AA1
:10151000145015101610171001E09394B0C114F078
:10152000B1C115F0B2C116F0B3C117F0010E141617
:10153000156A166A176A145015101610171001E074
:101540009396B0C114F0B1C115F0B2C116F0B3C199
:1015500017F0010E1416156A166A176A1450151042
:101560001610171001E09398B0C114F0B1C115F036
:10157000B2C116F0B3C117F0010E1416156A166A3F
:10158000176A145015101610171001E0939AB0C185
:1015900014F0B1C115F0B2C116F0B3C117F0010ECD
:1015A0001416156A166A176A1450151016101710BB
:1015B00001E0939CB0C114F0B1C115F0B2C116F0B6
:1015C000B3C117F0010E1416156A166A176A145083
:1015D00015101610171001E0939EB0C114F0B1C1A0
:1015E00015F0B2C116F0B3C117F0010E1416156A4A
:1015F000166A176A145015101610171001E096900D
:10160000B0C114F0B1C115F0B2C116F0B3C117F0FA
:10161000010E1416156A166A176A14501510161062
:10162000171001E09490B0C114F0B1C115F0B2C12F
:1016300016F0B3C117F0010E1416156A166A176A70
:10164000145015101610171001E09492B0C114F048
:10165000B1C115F0B2C116F0B3C117F0010E1416E6
:10166000156A166A176A145015101610171001E043
:101670009494B0C114F0B1C115F0B2C116F0B3C169
:1016800017F0010E1416156A166A176A1450151011
:101690001610171001E0949CB0C114F0B1C115F000
:1016A000B2C116F0B3C117F0010E1416156A166A0E
:1016B000176A145015101610171001E0949EB0C14F
:1016C00014F0B1C115F0B2C116F0B3C117F0010E9C
:1016D0001416156A166A176A14501510161017108A
:1016E00001E09590B0C114F0B1C115F0B2C116F08F
:1016F000B3C117F0010E1416156A166A176A145052
:1017000015101610171001E09592B0C114F0B1C178
:1017100015F0B2C116F0B3C117F0010E1416156A18
:10172000166A176A145015101610171001E09594D8
:10173000B0C114F0B1C115F0B2C116F0B3C117F0C9
:10174000010E1416156A166A176A14501510161031
:10175000171001E09596B0C114F0B1C115F0B2C1F7
:1017600016F0B3C117F0010E1416156A166A176A3F
:10177000145015101610171001E09598B0C114F010
:10178000B1C115F0B2C116F0B3C117F0010E1416B5
:10179000156A166A176A145015101610171001E012
:1017A000959AB0C114F0B1C115F0B2C116F0B3C131
:1017B00017F0010E1416156A166A176A14501510E0
:1017C0001610171001E0959CB0C114F0B1C115F0CE
:1017D000B2C116F0B3C117F0010E1416156A166ADD
:1017E000176A145015101610171001E0959EB0C11D
:1017F00014F0B1C115F0B2C116F0B3C117F0010E6B
:101800001416156A166A176A145015101610171058
:1018100001E09692B0C114F0B1C115F0B2C116F05A
:10182000B3C117F0010E1416156A166A176A145020
:1018300015101610171001E096943BD2B0C114F0A9
:10184000B1C115F0B2C116F0B3C117F0010E1416F4
:10185000156A166A176A145015101610171001E051
:101860009280B0C114F0B1C115F0B2C116F0B3C18D
:1018700017F0010E1416156A166A176A145015101F
:101880001610171001E09282B0C114F0B1C115F02A
:10189000B2C116F0B3C117F0010E1416156A166A1C
:1018A000176A145015101610171001E09284B0C179
:1018B00014F0B1C115F0B2C116F0B3C117F0010EAA
:1018C0001416156A166A176A145015101610171098
:1018D00001E09286B0C114F0B1C115F0B2C116F0AA
:1018E000B3C117F0010E1416156A166A176A145060
:1018F00015101610171001E09288B0C114F0B1C194
:1019000015F0B2C116F0B3C117F0010E1416156A26
:10191000166A176A145015101610171001E0928AF3
:10192000B0C114F0B1C115F0B2C116F0B3C117F0D7
:10193000010E1416156A166A176A1450151016103F
:10194000171001E09380B0C114F0B1C115F0B2C11D
:1019500016F0B3C117F0010E1416156A166A176A4D
:10196000145015101610171001E09382B0C114F036
:10197000B1C115F0B2C116F0B3C117F0010E1416C3
:10198000156A166A176A145015101610171001E020
:101990009384B0C114F0B1C115F0B2C116F0B3C157
:1019A00017F0010E1416156A166A176A14501510EE
:1019B0001610171001E09386B0C114F0B1C115F0F4
:1019C000B2C116F0B3C117F0010E1416156A166AEB
:1019D000176A145015101610171001E09388B0C143
:1019E00014F0B1C115F0B2C116F0B3C117F0010E79
:1019F0001416156A166A176A145015101610171067
:101A000001E0938AB0C114F0B1C115F0B2C116F073
:101A1000B3C117F0010E1416156A166A176A14502E
:101A200015101610171001E0938CB0C114F0B1C15D
:101A300015F0B2C116F0B3C117F0010E1416156AF5
:101A4000166A176A145015101610171001E0938EBD
:101A5000B0C114F0B1C115F0B2C116F0B3C117F0A6
:101A6000010E1416156A166A176A1450151016100E
:101A7000171001E09680B0C114F0B1C115F0B2C1E9
:101A800016F0B3C117F0010E1416156A166A176A1C
:101A9000145015101610171001E09480B0C114F006
:101AA000B1C115F0B2C116F0B3C117F0010E141692
:101AB000156A166A176A145015101610171001E0EF
:101AC0009482B0C114F0B1C115F0B2C116F0B3C127
:101AD00017F0010E1416156A166A176A14501510BD
:101AE0001610171001E09484B0C114F0B1C115F0C4
:101AF000B2C116F0B3C117F0010E1416156A166ABA
:101B0000176A145015101610171001E0948CB0C10C
:101B100014F0B1C115F0B2C116F0B3C117F0010E47
:101B20001416156A166A176A145015101610171035
:101B300001E0948EB0C114F0B1C115F0B2C116F03D
:101B4000B3C117F0010E1416156A166A176A1450FD
:101B500015101610171001E09580B0C114F0B1C136
:101B600015F0B2C116F0B3C117F0010E1416156AC4
:101B7000166A176A145015101610171001E0958296
:101B8000B0C114F0B1C115F0B2C116F0B3C117F075
:101B9000010E1416156A166A176A145015101610DD
:101BA000171001E09584B0C114F0B1C115F0B2C1B5
:101BB00016F0B3C117F0010E1416156A166A176AEB
:101BC000145015101610171001E09586B0C114F0CE
:101BD000B1C115F0B2C116F0B3C117F0010E141661
:101BE000156A166A176A145015101610171001E0BE
:101BF0009588B0C114F0B1C115F0B2C116F0B3C1EF
:101C000017F0010E1416156A166A176A145015108B
:101C10001610171001E0958AB0C114F0B1C115F08B
:101C2000B2C116F0B3C117F0010E1416156A166A88
:101C3000176A145015101610171001E0958CB0C1DA
:101C400014F0B1C115F0B2C116F0B3C117F0010E16
:101C50001416156A166A176A145015101610171004
:101C600001E0958EB0C114F0B1C115F0B2C116F00B
:101C7000B3C117F0010E1416156A166A176A1450CC
:101C800015101610171001E09682B0C114F0B1C102
:101C900015F0B2C116F0B3C117F0010E1416156A93
:101CA000166A176A145015101610171001E0968462
:101CB00000D0A66B00D0A52B3CEF04F01200808072
:101CC0008082808480868088808A818081828184ED
:101CD00081868188818A818C818E848012008280B5
:101CE00082828284828C828E8380838283848386B4
:101CF0008388838A838C838E848284841200D9CFE4
:101D0000E6FFE1CFD9FFE652DF6A804F8090814F36
:101D10008092824F8094834F8096844F8098854F25
:101D2000809A864F8190874F8192884F8194894F06
:101D300081968A4F81988B4F819A8C4F819C8D4FD1
:101D4000819E8E4F8490D768EE0ED66EF29401017C
:101D5000F451020A11E0030A09E0010A01E011D07E
:101D6000B6EC14F00101010EF46F0DD0D5EC14F0B7
:101D70000101020EF46F07D012EC10F00101F46BB8
:101D800002D00101F46BF2A4FED7DF2ADF50BDE1DF
:101D9000E552E552E7CFD9FF1200040120511F0B95
:101DA000010801E05BD02051600BE842E842E842C4
:101DB000E842E842010801E051D0245103E0240543
:101DC00001E04CD02151230A48E0010A40E0030A17
:101DD00030E0010A25E0240A22E0070A1FE0010A98
:101DE0001CE0030A11E0010A01E038D00101030EF2
:101DF000E76F0101D40EE86F010EE96F0101EF9367
:101E00000101080EEC6F2AD00101030EE76F0101FA
:101E1000D40EEA6F010EEB6F21D020D01FD01ED060
:101E20000101030EE76F0101C90EEA6F010EEB6FAE
:101E300015D00101030EE76F0101C90EE86F010E15
:101E4000E96F0101EF930101070EEC6F07D001016B
:101E5000030EE76F22C4D0F101D000D012000101BF
:101E6000C96BC20ECA6F010ECB6FCC6BCD6BCE6B44
:101E7000080ECF6FC26BC16B1A0E726E1E0E736EA0
:101E80000401000E166F050E176F400E146F04014B
:101E9000196F400E1A6F050E1B6F880E186F040124
:101EA000800E1E6F050E1F6F400E1C6F1200D9CFE3
:101EB000E6FFE1CFD9FF0101C16B040118BF30D0AB
:101EC000FC0EDBCF14F01951D880145403E2FC0E41
:101ED00019C4DBFF0101C16BFC0EDB50C15D19E2CF
:101EE000C151EA6A400FE96E050EEA22EF50E66E34
:101EF000C151E76EFD0EDBCFE9FFFE0EDBCFEAFF3F
:101F0000E750E926000EEA22E552E750EF6EC12BBA
:101F1000E3D70401400E196F1817187D880E1813A7
:101F20000101C15100D0E552E7CFD9FF1200D9CF4E
:101F3000E6FFE1CFD9FFE6520101C25101E02FD007
:101F4000DF6ADF2ADF50146E156AFF0E141801E1F4
:101F5000155001E10BD0FD0EDBCFE9FFDB2AFE0EB1
:101F6000DBCFEAFF01E3DB2AEF50EBE1DF50146E39
:101F7000156AD950FD0FE96EFF0EDA20EA6E145093
:101F8000EE5E1550ED5AFD0EDBCFC3F1FE0EDBCF3A
:101F9000C4F1DFCFC7F10101C86B010EC26FE5527A
:101FA000E552E7CFD9FF1200D9CFE6FFE1CFD9FF45
:101FB000E6520101C25101E030D0DF6ADF2ADF5072
:101FC000146E156AFF0E141801E1155001E10CD0D2
:101FD000FD0EDBCFF6FFDB2AFE0EDBCFF7FF01E3C2
:101FE000DB2A0800F550EAE1DF50146E156AD9507B
:101FF000FD0FE96EFF0EDA20EA6E1450EE5E15500A
:10200000ED5AFD0EDBCFC3F1FE0EDBCFC4F1DFCF07
:10201000C7F10101010EC86FC26FE552E552E7CF6B
:10202000D9FF1200D9CFE6FFE1CFD9FFE652040174
:102030001CBF6BD0030E0101C25D01E1C26BC25136
:1020400001E163D0020EC25D06E104011D6B0101D6
:10205000030EC26F54D0C20552E1400E146E156AD1
:10206000C751145C000E155803E2400EDF6E02D01B
:10207000C7C1DFFFDFCF1DF4DF50C75DC76F800E24
:10208000C56F050EC66FC80515E1DF5012E0C3C16C
:10209000F6FFC4C1F7FF0800F550C5C1E9FFC6C18E
:1020A000EAFFEF6EC52B000EC623C32BC423DF0649
:1020B000ECD713D0DF5011E0C3C1E9FFC4C1EAFF80
:1020C000EF50C5C1E9FFC6C1EAFFEF6EC52B000E98
:1020D000C623C32BC423DF06EDD7C75110E104018B
:1020E0001D51146E156A400E141801E1155004E1DB
:1020F0000101020EC26F03D00101030EC26F400E38
:1021000004011C171C7D880E1C13E552E552E7CF15
:10211000D9FF120004012051600BE842E842E84276
:10212000E842E842000901E055D02151070A51E098
:102130000B0A4FE0070A40E0010A2CE00B0A28E0F6
:10214000020A26E0030A22E0080A12E0010A0EE071
:102150000F0A0AE0030A01E03CD00101010EE76F1B
:102160000101040EEE6F36D036D834D090D832D07C
:102170000101010EE76F0101F00EE86F010EE96F3A
:102180000101EF930101010EEC6F24D0A8D822D0F9
:10219000F4D820D00101010EE76F040124510101A0
:1021A000E86FE96BF10EE827010EE9230101EF93D7
:1021B0000101010EEC6F0ED00101010EE76F040169
:1021C0002451EA6AF10FE96E010EEA2222C4EFFF00
:1021D00001D000D01200800E0401205D57E1235190
:1021E000030A34E0010A10E0030A01E04DD00101C6
:1021F000010EE76F0101D20EE86F2B0EE96F120E90
:102200000101EC6FED6B40D00101010EE76F04019D
:102210002251F66EF76AD890F636F736930EF62608
:102220002C0EF7220900F5CFE8F10A00F5CFE9F10D
:10223000020E0101F76AE825F66EE951F72209005E
:10224000F5CFECF10A00F5CFEDF11ED00101010E42
:10225000E76F04012251F66EF76AD890F636F7362A
:10226000970EF6262C0EF7220900F5CFE8F10A00AA
:10227000F5CFE9F1E8C1F6FFE9C1F7FF0800F55035
:102280000101EC6FED6B00D00101EF831200010141
:10229000010EE76F0F0EE66E710EE66E0F0EE66E24
:1022A0005FEC15F0E552E552E552010EE66EF10ED7
:1022B000E66E010EE66E5FEC15F0E552E552E55272
:1022C00022C4F0F10401225104E10101050EEE6F78
:1022D00005D00101060EEE6F2FEC0FF01200040185
:1022E000606B616B040120511F0B020A14E0030AAA
:1022F0000EE0010A01E033D00101010EE76F040195
:1023000060810101EFA102D00401608328D00101A6
:10231000010EE76F24D00101010EE76F0401245183
:102320000F0B080DF350156A000F146E040E1522E2
:102330002451800B01E0010E040DF350010114241F
:10234000EA6F000E1520EB6FEAC1E9FFEBC1EAFF6F
:10235000EF50040B03E00401010E606F00D0010197
:10236000E7050AE10101600EE86F040EE96F010163
:10237000EF930101020EEC6F12000401220510E13F
:1023800020511F0B00090CE10101010EE76F030E44
:102390000401215D03E10101EF8102D00101EF9110
:1023A000040122513AE120511F0B020836E1245169
:1023B0000F0B000932E00101010EE76F0401245107
:1023C0000F0B080DF350156A000F146E040E152242
:1023D0002451800B01E0010E040DF350010114247F
:1023E000EA6F000E1520EB6F030E0401215D07E17B
:1023F000840EEAC1E9FFEBC1EAFFEF6E0ED024AF15
:1024000006D0EAC1E9FFEBC1EAFFEF6A06D0880E09
:10241000EAC1E9FFEBC1EAFFEF6E12006C5002E087
:10242000000E01D0010E00090BE0040100513C0B2D
:10243000E842E8420D0802E10CD801D040D808D0AB
:102440006C5002E0000E01D0010E040901E047D8F3
:102450001200D9CFE6FFE1CFD9FFE6520101E66BCA
:10246000E76BEC6BED6B8AEC10F0DF6ADF50146EFB
:10247000156A010E145C000E15581BE20101E751AC
:1024800001E017D0F76ADF34FE0BF736F66E9D0ECB
:10249000F6262C0EF7220900F5CF14F00800F5CF30
:1024A00015F004D015C0FAFF1450F96EFBDFDF2AD7
:1024B000DDD7DDD8E552E552E7CFD9FF1200020E95
:1024C0000101E65D0AE196D8040100BD03D0C80E03
:1024D000006F02D0880E006F01D00FD91200040ED9
:1024E0000101EE5D0AE122C46EFF6E50000803E2B6
:1024F000050EEE6F02D0030EEE6F0101E6050AE154
:102500000BD8040104BD03D0C80E046F02D0880E9E
:10251000046F01D0F2D81200D9CFE6FFE1CFD9FF86
:10252000020EE1260101400EEC5D000EED5905E2C0
:10253000ECC1DEFFEDC1DDFF03D0400EDE6EDD6AD3
:10254000040104930491010EDB500413DFCF05F462
:10255000000EDB500101EC5F010EDB50ED5B600E05
:10256000EA6F040EEB6F0101EFA31ED0D9CFE9FF94
:10257000DACFEAFFEE50ED1016E0E8C1F6FFE9C150
:10258000F7FF0800F550EAC1E9FFEBC1EAFFEF6E83
:102590000101EA2B000EEB23E82BE923DF06010EF5
:1025A00001E2DB06E3D71CD0D9CFE9FFDACFEAFF9F
:1025B000EE50ED1015E0E8C1E9FFE9C1EAFFEF5088
:1025C000EAC1E9FFEBC1EAFFEF6E0101EA2B000E61
:1025D000EB23E82BE923DF06010E01E2DB06E4D75B
:1025E000020EE15C02E2E16AE552E16EE552E7CFFC
:1025F000D9FF1200D9CFE6FFE1CFD9FF020EE126C5
:10260000030E04010015E76E010EE7CFDBFF01C4E6
:10261000DFFFDE500101EC27DD50ED23600EE86F97
:10262000040EE96FD9CFE9FFDACFEAFFEE50ED10E3
:1026300014E0E8C1E9FFE9C1EAFFEF50EAC1E9FFB0
:10264000EBC1EAFFEF6EEA2B000EEB23E82BE92348
:10265000DF06010E01E2DB06E5D7020EE15C02E2D5
:10266000E16AE552E16EE552E7CFD9FF12000101C0
:10267000E7510CE10401400E016F200E026F040EC1
:10268000036F840E006F0401046F35D0040120AF86
:1026900022D00101EC510401265D0101ED5104013C
:1026A000275904E226C4ECF127C4EDF135DF01011E
:1026B000010EE66F0401400E016F200E026F040E42
:1026C000036F800E006F0401600E066F040E076F2B
:1026D000C80E046F10D00101020EE66F0401056BF5
:1026E000C80E046F0401400E016F600E026F040EED
:1026F000036FC80E006F6D9812000101E66B0401B4
:10270000400E016F200E026F040E036F880E006FE3
:102710000401046B12000F9E05D00F9E07AE02D07D
:10272000076C0F8E07C001F0006A136A126A860EEA
:10273000026E036A4CEF14F00F6A88EC14F0A0EC00
:1027400014F00FB630EF14F00FA205D00FB830EF31
:1027500014F037EF14F00FAA05D00FB030EF14F0DB
:1027600037EF14F00FB002D00FA802D043EF14F0EF
:10277000036A0D500824026EE86A03227E0E025E90
:10278000E86A035A126A136A006A016A0C50070267
:10279000F4CF01F0F3CF00F00B500702F3501326F3
:1027A000F4500022000E01220C500602F3501326B2
:1027B000F4500022000E01220A500702F3501226A4
:1027C000F4501322000E002201220B500602F35097
:1027D0001226F4501322000E002201220C50050292
:1027E000F3501226F4501322000E002201220A5048
:1027F0000602F4501226000E1322002201220B5072
:102800000502F4501226000E1322002201224CEF82
:1028100014F00F6A88EC14F00FB613EF14F00FA247
:102820000AD00FB403D07F0E076E19D0800E076E4A
:1028300016D0076A14D00FB0FCD7870E0860F1D706
:102840007E0E0864F6D7860E085C04E0D890073246
:10285000082AF9D70FA403D0076C07AEEAD71200F5
:102860007F0E086EFF0E076E066E056E12007F0E5D
:102870000FBEFF0E086E02D07F0E086E800E076E30
:10288000066A056AF3D70FAE04D0800E086E076A99
:10289000F7D7086A076AF4D7015000101310121016
:1028A000F8E003BEF0D701BE0CD002500310EBE0FD
:1028B000D89012361336003601360206D8A0030629
:1028C000F2D70350D4E10228D2E012AE11D07F0E2D
:1028D000121402E113A00CD0132AE86A002201228C
:1028E00007E3D880013200321332022A0228BFE007
:1028F0000250C9E013C005F000C006F00134076EB5
:102900000230086E0732089E0FBE088E36EF14F0B4
:102910000736083602E30F840F7E06E10F80086A4F
:10292000076A066A056A1200082803E0D8800732A1
:102930001200D890073202E10F8212000F861200B7
:102940000C360D3602E30F8C0F7E06E10F880D6A00
:102950000C6A0B6A0A6A12000D2803E0D8800C3258
:102960001200D8900C32EAE10F8A12006DA60FD83F
:1029700002D06DB613D80101EE0508E16DBA06D09C
:10298000686A696A69806988020EEE6F12006D6A72
:10299000696A6D860101010EEE6F12006D6A696A47
:1029A0000101EE6B1200CEEF14F00101EE5101E1D6
:1029B0003AD06850040B04E06950040B01E03CD8A5
:1029C0006DB231D06850010B04E06950010B01E099
:1029D00054D86850100B04E06950100B01E024D863
:1029E0006850400B04E06950400B01E03BD8685050
:1029F000200B04E06950200B01E036D86850020B30
:102A000004E06950020B01E036D8030E0101EE5DCF
:102A100001E209D06850080B06E06950080B03E09A
:102A20000EEC12F068961200698468986D82A19A83
:102A3000A08A0300A09A12006D9269946894120013
:102A40000101EFA10ED0F8DF6D840101080EF26FD5
:102A5000070EF36FF207000EF35BF251F311FAE188
:102A60006D941200689C120070A003D07DEC13F0EE
:102A70007090689A1200689212006A6A686A9F0EE3
:102A80006B6E7B0E696E6E6A0F0EE66E710EE66EF1
:102A90000F0EE66E14D8E552E552E552160E706E32
:102AA00068A602D06896FCD76D987DEC13F0010102
:102AB000EF910101F06B0101030EEE6F1200D9CF0F
:102AC000E6FFE1CFD9FFFD0EDBCFE9FFFE0EDBCF46
:102AD000EAFFFC0EDB5004E0EE6AFC0EDB06F9D7E1
:102AE000E552E7CFD9FF1200FF0EE3CFEAFFE55230
:102AF000FF0EE3CFE9FFE552E66AE66AD9CFE6FFCB
:102B0000DACFE6FFFC0EE124D96EFF0EE220DA6E8A
:102B1000E66AE66AE66A200EEF5C06E0090EEF5C04
:102B200003E0EF6603D03FD0EE50F5D72D0EEF5CFB
:102B300003E1FF0EE32A03D02B0EEF5C01E1EE5020
:102B40002F0EEF6424D03A0EEF6021D0D890F90E0A
:102B5000E336FA0EE336FD0EDECFE3FFFE0EDDCFE9
:102B6000E3FFD890F90EE336FA0EE336D890F90E6B
:102B7000E336FA0EE336FD0EE350DE26FE0EE3509A
:102B8000DD22300EEE5CDE26000EDD22D9D7FF0EF0
:102B9000E3CFE8FFE85207E0F90EE31EE32AFA0E5E
:102BA000D8B4E306E31EE552E552E552FF0EE3CF4B
:102BB000DAFFE552FF0EE3CFD9FFE552E1CFE9FF9F
:102BC000E2CFEAFFED52ED52EECFF3FFEFCFF4FF8D
:102BD00012001201000202000040D8040A000000A6
:102BE00001020001090243000201008032090400D1
:102BF0000001020201000524001001042402020564
:102C0000240600010524010001070582034000029B
:102C100009040100020A0000000705030240000049
:102C2000070583024000000403090434034D0069D2
:102C300000630072006F006300680069007000208C
:102C40000054006500630068006E006F006C006F48
:102C50000067007900200049006E0063002E0034F8
:102C6000034300440043002000520053002D003273
:102C70000033003200200045006D0075006C0061DB
:102C800000740069006F006E002000440065006D54
:102C9000006F00E42BE42B272C2B2C5F2C9A1DFFBC
:102CA000D9CFE6FFE1CFD9FF550EE12630D8010E8E
:102CB000D56ED58E40D8060E0101EE5D1DE36D5038
:102CC000020B1AE1380ED76EC70ED66EF294F2B42C
:102CD00004D031D81FEC04F0FAD75FEC0EF0FC0EF4
:102CE000D76EF90ED66EF294F2B404D024D81FEC4D
:102CF00004F0FAD77FEC0EF0DDD7550EE15C02E26E
:102D0000E16AE552E16EE552E7CFD9FF1200C26AEF
:102D10000F0EC16EB468656A926A936A946A956A86
:102D2000966A140E6F6E0101EE6B0101EF6B0101EB
:102D3000F06B1CEF04F084828484B6EC14F084946D
:102D4000D5EC14F0848412EC10F084948492120078
:102D50002A0EF66E080EF76E000EF86E01010900DD
:102D6000F550E16F0900F550E26F03E1E16701D032
:102D70003DD00900F550DC6F0900F550DD6F09000A
:102D8000F550DE6F09000900F550E96E0900F550B5
:102D9000EA6E090009000900F550DF6F0900F550DF
:102DA000E06F09000900F6CFE3F1F7CFE4F1F8CFC7
:102DB000E5F1DCC1F6FFDDC1F7FFDEC1F8FF01017F
:102DC000DF5302E1E05307E00900F550EE6EDF0744
:102DD000F8E2E007F9D7E3C1F6FFE4C1F7FFE5C188
:102DE000F8FF0101E107000EE25BBFD71200504976
:102DF00043313846343535302046756C6C2D537070
:102E000065656420555342202D204344432052538E
:102E10002D32333220456D756C6174696F6E2044BC
:102E2000656D6F0D0A0D0A001B5B324A000013EE40
:102E300000F023EE00F0F86A0F9CA8EC16F02CECE2
:102E400017F050EC16F0FBD7120000EE00F00F0E5A
:102E5000EE6AEA62FDD712001200FFFFFFFFFFFFDC
:102E6000FFFFFFFFFFFFFFFFFFFFFFFFFFFFFFFF72
:102E7000FFFFFFFFFFFFFFFFFFFFFFFFFFFFFFFF62
:102E8000FFFFFFFFFFFFFFFFFFFFFFFFFFFFFFFF52
:102E9000FFFFFFFFFFFFFFFFFFFFFFFFFFFFFFFF42
:0200000400F00A
:020000040030CA
:0E000000220F391E008180000FC00FE00F405C
:020000040020DA
:08000000FFFFFFFFFFFFFFFF00
:00000001FF
